:03000000020120DA
:10002B0002015CE627F60809E637F60809E637F61B
:10003B001818191922C3E697F60809E697F6080966
:10004B00E697F61818191922C3ED33FDEE33FEEFC0
:10005B0033FFEA33FAEB33FBEC33FC22E633F608DF
:10006B00E633F608E633F6181822E6FD08E6FE0836
:10007B00E6FF18187A007B007C0075F0181153C34B
:10008B00EA9709EB9709EC971919B3500FC3EA9745
:10009B00FA09EB97FB09EC97FC1919B31167D5F02B
:1000AB00DC22E7F5F0E6A4FAABF009E7F5F0E6A4FD
:1000BB002BFBE5F03CFC09E7F5F0E6A42CFC191949
:1000CB0008E7F5F0E6A42BFBE5F03CFC08E7F5F0C0
:1000DB00E6A42CFC0918E7F5F0E6A42CFC1908ECB7
:1000EB00F618EBF618EAF622E6F70809E6F7080920
:1000FB00E6F722C230C231C232C233C234753C0081
:10010B00753D00753E00753F00753B00756B0075C6
:10011B003037020120C2927581E0E530B437D475D7
:10012B0030C8753A0A75C90075C80475CAF075CB25
:10013B00D8758DFE7589297587807598D07588550A
:10014B0075B80375A8A0020A6075A8007530372131
:10015B0020C0D0D2D3C2D4C0E0B2B6C2CF153A20A1
:10016B00310912018C1208F71203C41202DC1203BC
:10017B000112032612034B120378C2CFD0E0D0D06A
:10018B00328525F0752500A2B5B39228A2B3B392A0
:10019B0029A295B3922AE5256003B5F00122302AF6
:1001AB005020300E053B74F8253B5045753B000243
:1001BB0001FCE53BB40005D2320201FCB40105D2CF
:1001CB00320201FCB40205D2320201FCB40305C2B7
:1001DB00300201FCB40405D2330201FCB40505D294
:1001EB00340201FCB40605D2340201FCB40702D27E
:1001FB003530286DD230E53BB40010E5422401D4F4
:10020B00F542B4240375420002026CB40110E543BD
:10021B002401D4F543B4320375430102026CB402DA
:10022B000AE5452401D4F54502026CB4040FE5350B
:10023B002401F535E5363400F53602026CB4050AB7
:10024B00E5382401D4F53802026CB4060AE53924EA
:10025B0001D4F53902026C056BE56BB40C03756BBD
:10026B000030296BD230E53BB40010E5412401D4BA
:10027B00F541B460037541000202DAB40110E544A4
:10028B002401D4F544B413037544010202DAB40219
:10029B00030202DAB40410E535C39401F535E536F3
:1002AB009400F5360202DAB4050AE5372401D4F5D9
:1002BB00370202DAB4060AE5382410D4F538020204
:1002CB00DAB4070BE56B245FF8E604F60202DA21D9
:1002DB00A8A21392A6A21292A4A21B92A2A21A9255
:1002EB00A0A21F92A1A21C92A3A21792A5A2149244
:1002FB00A7C291D29122A21592A7A21692A5A21DD6
:10030B0092A3A21E92A1A21992A0A21892A2A2112C
:10031B0092A4A21092A6C290D29022A20392A0A263
:10032B000292A2A20B92A4A20A92A6A20F92A7A239
:10033B000C92A5A20792A3A20492A1C297D29722D4
:10034B00A20592A1A20692A3A20D92A5A20E92A71C
:10035B00A20992A6A20892A4A20192A2A20092A024
:10036B00C2B2D2B222010204081020408090037066
:10037B00E53B93F4F524A2209287A2219286A22238
:10038B009280A2239281A2249282A2259283A226FA
:10039B009284A227928522C0F9A4B0999282F88008
:1003AB00908883C6A1868E4079243019120278007A
:1003BB001008034621060EBFFF783C79207A049083
:1003CB0003A2E69320B601F4F70809DAF222753A94
:1003DB000A3099FDA2D0929BF599C29922753A0ADF
:1003EB00E53A60113098F9E59920D006209A06027B
:1003FB000404209A04D3020405C3C29822D3020436
:10040B007F71E840F8B4EFF571E840F1B4F3EE71A9
:10041B00E840EAF53171E840E4F53271E840DEF589
:10042B003371E840D8F53471E840D2203002F5350D
:10043B0071E840C9203002F53671E840C020300227
:10044B00F53771E840B7203002F53871E840AE203F
:10045B003002F53971E840A5F5527853790C71E803
:10046B00409BF608D9F8790C71E84091203001F6E1
:10047B0008D9F5C322D29974EF71D974F371D9A944
:10048B006F7870E671D908D9FAC2312200000000EA
:10049B000000406F14008D2740FC3BC0C24F003260
:1004AB006480F877C0678C00D7A0000000000000C4
:1004BB00000000000000000000000000809DB4C0A0
:1004CB000CC940D3DC000000000000C0A800805124
:1004DB000140FA0100A302C04B0380F403409D04CA
:1004EB0000460500000000000000000000000000B6
:1004FB000000000000C0EE0580970640400700E9B1
:10050B0007C09108803A0940E309008C0AC0340BFC
:10051B0080DD0B0000000000000000000000000068
:10052B00000000000040860C002F0DC0D70D80800E
:10053B000E40290F00D20FC07A1080231140CC112E
:10054B000075120000000000000000000000000019
:10055B000000000000C01D1380C613000000080738
:10056B0000100E00181500201C00282300302A0054
:10057B00383100403800483F000000000000000008
:10058B000000000000000000000000504600584D25
:10059B0000605400685B0070620078690080700036
:1005AB00887700907E009885000000000000000016
:1005BB000000000000000000000000A08C00A893C9
:1005CB0000B09A00B8A1000000001E00003C000023
:1005DB005A0000780000960000B40000D20000F032
:1005EB0000000E01000000000000000000000000F1
:1005FB00000000000000002C01004A01006801000F
:10060B00860100A40100C20100E00100FE01001CF4
:10061B0002003A0200000000000000000000000091
:10062B000000000000000058020076020094020057
:10063B00B20200D00200EE02000C03002A030048B5
:10064B000300660300000000000000000000000033
:10065B0000000000000000840300A20300C00300A0
:10066B00DE0300FC03001A04003804005604007477
:10067B0004009204000000000000000000000000D5
:10068B0000000000000000B00400CE0400EC0400E9
:10069B000A0500280500460500640500820500A038
:1006AB000500BE0500000000000000000000000077
:1006BB0000000000000000DC0500FA050018060031
:1006CB00360600540600720600900600AE0600CCFB
:1006DB000600EA0600000001010202030304040005
:1006EB0000000000000505060607070808090900B9
:1006FB0000000000000A0A0B0B0C0C0D0D0E0E0077
:10070B0000000000000F0F10101111121213130034
:10071B0000000000001414151516161717181800F2
:10072B00000000000019191A1A1B1B1C1C1D1D753B
:10073B004600754700754800E54475F003A4900426
:10074B00972582F582E5F03583F5837849E493F6B6
:10075B0008740193F608740293F678467949112EC2
:10076B00E54375F003A49004D02582F582E5F035BE
:10077B0083F5837849E493F608740193F6087402C1
:10078B0093F678467949112EE54275F003A490054E
:10079B00662582F582E5F03583F5837849E493F697
:1007AB0008740193F608740293F678467949112E72
:1007BB00E54175F003A49005D22582F582E5F0356D
:1007CB0083F5837849E493F608740193F608740271
:1007DB0093F678467949112EE5409006E0784993D7
:1007EB00F608E4F608F678467949112E75497F75B7
:1007FB004A42754BF1784979461200407849794F56
:10080B001200F378707401F608E54FF608E550F620
:10081B0008E551F608E545540FF9E545C4540F7545
:10082B00F00AA429F6D231756F05C232221F1D1FA3
:10083B001E1F1E1F1F1E1F1E1FC2AF7846747FF682
:10084B00087442F60874F1F6784679311200407557
:10085B00491E754A00754B0078467949120075EAB6
:10086B0075F00584C4C5F02325F0F54075493C753A
:10087B004A00754B0078467949120075EA75F00A03
:10088B0084C425F0F541754918754A00754B0078FD
:10089B00467949120075EA75F00A84C425F0F542D1
:1008AB00E53475F00A84D4C454F025F0F545AA4616
:1008BB00AB477C00C3EC90083893F5F0EA95F0EB6E
:1008CB009400400BEA95F0FAEB9400FB0C01BFECA3
:1008DB000475F00A84C454F025F0F544EA0475F06D
:1008EB000A84C454F025F0F543D2AF22E53BB400A3
:1008FB001FE542540F4410F53DE542C4540FF53C3F
:10090B00E541540FF53FE541C4540FF53E020A197A
:10091B00B4011FE543540F4410F53DE543C4540F98
:10092B00F53CE544540FF53FE544C4540FF53E0246
:10093B000A19B4021FE545540F4410F53DE545C4B3
:10094B00540FF53CE540540FF53FE540C4540FF50B
:10095B003E020A19B40319E55275F0058485F03D82
:10096B0075F00584F53F85F03E7421F53C020A19BC
:10097B00B4041DE535540FF53FE535C4540FF53E72
:10098B00E536540FF53DE536C4540FF53C020A1914
:10099B00B40519E537540FF53FE537C4540FF53E51
:1009AB00E538540FF53D753C21020A19B4061AE5DA
:1009BB0039540FF53EE539C4540FF53DE538C454B1
:1009CB000FF53F753C21020A19B40738E56B047526
:1009DB00F00A84F53C43F01085F03D7453256BF819
:1009EB00E6F5F0740C28F8E6A433E5F03350057403
:1009FB0078F621D7F5F0540FF53FE5F0C4540FF519
:100A0B003E020A197420F53CF53DF53EF53F227880
:100A1B00707402F608E535F608E536F6756F03C215
:100A2B0033D2312278707403F608E537F608E538CF
:100A3B00F608E539F6756F04C234D231227870743A
:100A4B0004F608795F7A0CE7F60809DAFA756F0D88
:100A5B00C235D2312212040C40FB2030021144303B
:100A6B00320AC2AF12073AD2AF020A8F30330551A6
:100A7B001A020A8F303405512F020A8F3035055177
:0E0A8B0048020A8F303105120480C2304160EB
:00000001FF
